:020000040000FA
:0408000054EF09F0B8
:1008100003B283EF05F0F2B4A1EF05F09EB0A9EFAB
:1008200005F09EB2B1EF05F0F2A81AEF04F0F2B2B3
:1008300032EF04F09EB61FEF04F003EF09F09E962E
:1008400000011350000A06E000011350010A06E0FF
:1008500003EF09F0DCEC1CF003EF09F0D0EC1EF024
:1008600003EF09F0CD90F2929EA03CEF04F001015D
:10087000533F3CEF04F0542BAEC1B2F1AFC1B3F122
:10088000B0C1B4F1B1C1B5F1AAC1AEF1ABC1AFF124
:10089000ACC1B0F1ADC1B1F1A6C1AAF1A7C1ABF134
:1008A000A8C1ACF1A9C1ADF1A2C1A6F1A3C1A7F144
:1008B000A4C1A8F1A5C1A9F19EC1A2F19FC1A3F154
:1008C000A0C1A4F1A1C1A5F19AC19EF19BC19FF164
:1008D0009CC1A0F19DC1A1F196C19AF197C19BF174
:1008E00098C19CF199C19DF1CECF96F1CFCF97F1F0
:1008F00053C198F154C199F1CF6ACE6A0101536B8B
:10090000546B9E90CD800FBC0F8E0FBA8BEF04F00E
:100910000F8A03EF09F00F8C0FBEC7EF04F096C1EA
:100920009AF197C19BF198C19CF199C19DF19AC12F
:100930009EF19BC19FF19CC1A0F19DC1A1F19EC1FF
:10094000A2F19FC1A3F1A0C1A4F1A1C1A5F1A2C1CF
:10095000A6F1A3C1A7F1A4C1A8F1A5C1A9F1A6C19F
:10096000AAF1A7C1ABF1A8C1ACF1A9C1ADF1AAC16F
:10097000AEF1ABC1AFF1ACC1B0F1ADC1B1F1AEC13F
:10098000B2F1AFC1B3F1B0C1B4F1B1C1B5F1010180
:100990005E6B5F6B606B616B96515E2797515F2357
:1009A00098516023995161239A515E279B515F238F
:1009B0009C5160239D5161239E515E279F515F236F
:1009C000A0516023A1516123A2515E27A3515F234F
:1009D000A4516023A5516123A6515E27A7515F232F
:1009E000A8516023A9516123AA515E27AB515F230F
:1009F000AC516023AD516123AE515E27AF515F23EF
:100A0000B0516023B1516123B2515E27B3515F23CE
:100A1000B4516023B5516123D89001016133603333
:100A20005F335E33D8900101613360335F335E33EF
:100A3000D8900101613360335F335E3300C10CF144
:100A400001C10DF102C10EF103C10FF104C110F19A
:100A500005C111F106C112F107C113F108C114F16A
:100A600009C115F10AC116F10BC117F134C135F1F5
:100A700011B846EF05F00101620E046F010E056F1B
:100A8000000E066F000E076F4FEF05F00101A70E75
:100A9000046F020E056F000E066F000E076F5EC139
:100AA00000F15FC101F160C102F161C103F173ECBA
:100AB0001BF003BF04D018BE02D018A0108C11A0E8
:100AC00067EF05F010BA67EF05F00F80108A0CC1D0
:100AD00000F10DC101F10EC102F10FC103F110C10E
:100AE00004F111C105F112C106F113C107F114C1DE
:100AF00008F115C109F116C10AF117C10BF135C191
:100B000034F103EF09F00392ABB2AB98AB88030169
:100B100003EE00F080517F0BE92604C0EFFF802B2D
:100B20008151805D700BD8A48B8200008051815D63
:100B3000700BD8A48B9281518019D8B4079003EF21
:100B400009F0F2940101453F03EF09F0462B03EF52
:100B500009F09E900101533F03EF09F0542B03EF7E
:100B600009F09E9211B819EF07F08BB4BFEF05F0B2
:100B700010ACBFEF05F08B84109CC0EF05F08B9498
:100B8000C3CF55F1C4CF56F1C28207B42AEF06F0A5
:100B900047C14BF148C14CF149C14DF14AC14EF139
:100BA0005EC162F15FC163F160C164F161C165F171
:100BB00096C1B6F197C1B7F198C1B8F199C1B9F131
:100BC0009AC1BAF19BC1BBF19CC1BCF19DC1BDF101
:100BD0009EC1BEF19FC1BFF1A0C1C0F1A1C1C1F1D1
:100BE000A2C1C2F1A3C1C3F1A4C1C4F1A5C1C5F1A1
:100BF000A6C1C6F1A7C1C7F1A8C1C8F1A9C1C9F171
:100C0000AAC1CAF1ABC1CBF1ACC1CCF1ADC1CDF140
:100C1000AEC1CEF1AFC1CFF1B0C1D0F1B1C1D1F110
:100C2000B2C1D2F1B3C1D3F1B4C1D4F1B5C1D5F1E0
:100C3000010155515B2756515C23E86A5D230E2E56
:100C40002AEF06F05CC157F15DC158F15B6B5C6B3C
:100C50005D6B078E0201002F03EF09F03C0E006F61
:100C600016AE108E00C10CF101C10DF102C10EF1E2
:100C700003C10FF104C110F105C111F106C112F158
:100C800007C113F108C114F109C115F10AC116F128
:100C90000BC117F134C135F101018A6757EF06F036
:100CA0008B6757EF06F08C6757EF06F08D675BEFA9
:100CB00006F08BEF06F08EC100F18FC101F190C1FB
:100CC00002F191C103F10101010E046F000E056FE5
:100CD000000E066F000E076F73EC1BF000C18EF163
:100CE00001C18FF102C190F103C191F1006780EF62
:100CF00006F0016780EF06F0026780EF06F00367F9
:100D00008BEF06F08AC18EF18BC18FF18CC190F10F
:100D10008DC191F10F80D57ED5BE6DD0D6CF47F174
:100D2000D7CF48F145C149F1E86AE8CF4AF118BE8A
:100D300002D018A0108C109047C100F148C101F1F9
:100D400049C102F14AC103F101010A0E046F000E0C
:100D5000056F000E066F000E076F73EC1BF003AFFC
:100D60001080010154A7C1EF06F00F9A0F9C0F9E4F
:100D70000101000E5E6F600E5F6F3D0E606F080E2A
:100D8000616F010147BFD1EF06F04867D1EF06F070
:100D90004967D1EF06F04A67D1EF06F0F288F6EF27
:100DA00006F0F2985E6B5F6B606B616B966B976B96
:100DB000986B996B9A6B9B6B9C6B9D6B9E6B9F6BFF
:100DC000A06BA16BA26BA36BA46BA56BA66BA76BAF
:100DD000A86BA96BAA6BAB6BAC6BAD6BAE6BAF6B5F
:100DE000B06BB16BB26BB36BB46BB56BD76AD66AD1
:100DF0000101456B466B0CC100F10DC101F10EC143
:100E000002F10FC103F110C104F111C105F112C1CA
:100E100006F113C107F114C108F115C109F116C19A
:100E20000AF117C10BF135C134F103EF09F003EFFB
:100E300009F00201002F6AEF08F0D59ED6CF47F1E6
:100E4000D7CF48F145C149F1E86AE8CF4AF1D76AFE
:100E5000D66A0101456B466BD58E108E16AE198C85
:100E600000C10CF101C10DF102C10EF103C10FF17E
:100E700004C110F105C111F106C112F107C113F14E
:100E800008C114F109C115F10AC116F10BC117F11E
:100E900034C135F10FA0109A11B85AEF07F00101D3
:100EA000620E046F010E056F000E066F000E076FD5
:100EB00063EF07F00101A70E046F020E056F000E2D
:100EC000066F000E076F47C100F148C101F149C12B
:100ED00002F14AC103F173EC1BF003BF76EF07F098
:100EE00018BE02D018A0108C11B00F800CC100F1F8
:100EF0000DC101F10EC102F10FC103F110C104F1E6
:100F000011C105F112C106F113C107F114C108F1B5
:100F100015C109F116C10AF117C10BF135C134F140
:100F200002013C0E006F00C10CF101C10DF102C1C4
:100F30000EF103C10FF104C110F105C111F106C199
:100F400012F107C113F108C114F109C115F10AC169
:100F500016F10BC117F134C135F101018A67B8EF01
:100F600007F08B67B8EF07F08C67B8EF07F08D6775
:100F7000BCEF07F0ECEF07F08EC100F18FC101F17B
:100F800090C102F191C103F10101010E046F000E45
:100F9000056F000E066F000E076F73EC1BF000C1AB
:100FA0008EF101C18FF102C190F103C191F100678F
:100FB000E1EF07F00167E1EF07F00267E1EF07F00B
:100FC0000367ECEF07F08AC18EF18BC18FF18CC102
:100FD00090F18DC191F10F80109047C100F148C18F
:100FE00001F149C102F14AC103F101010A0E046F86
:100FF000000E056F000E066F000E076F73EC1BF0FE
:1010000003AF1080010154A712EF08F00F9A0F9C54
:101010000F9E0101000E5E6F600E5F6F3D0E606FF0
:10102000080E616F47C100F148C101F149C102F1E9
:101030004AC103F10101140E046F050E056F000E85
:10104000066F000E076F73EC1BF003AF2BEF08F079
:10105000F28850EF08F0F2985E6B5F6B606B616B2B
:10106000966B976B986B996B9A6B9B6B9C6B9D6B5C
:101070009E6B9F6BA06BA16BA26BA36BA46BA56B0C
:10108000A66BA76BA86BA96BAA6BAB6BAC6BAD6BBC
:10109000AE6BAF6BB06BB16BB26BB36BB46BB56B6C
:1010A0000CC100F10DC101F10EC102F10FC103F13C
:1010B00010C104F111C105F112C106F113C107F10C
:1010C00014C108F115C109F116C10AF117C10BF1DC
:1010D00035C134F18FEC1FF01A661ED019AE11D055
:1010E000199E1A8E17AE07D0136A040E146E156A75
:1010F000DCEC1CF011D0136A146A156ADCEC1CF0ED
:101100000BD019AC09D0199C1A8C010E136E146AFD
:10111000156AD0EC1EF000D08BB496EF08F010AC3E
:1011200096EF08F08B84109C97EF08F08B94C3CF58
:1011300055F1C4CF56F1C28207B401EF09F047C19F
:101140004BF148C14CF149C14DF14AC14EF15EC16C
:1011500062F15FC163F160C164F161C165F196C183
:10116000B6F197C1B7F198C1B8F199C1B9F19AC177
:10117000BAF19BC1BBF19CC1BCF19DC1BDF19EC147
:10118000BEF19FC1BFF1A0C1C0F1A1C1C1F1A2C117
:10119000C2F1A3C1C3F1A4C1C4F1A5C1C5F1A6C1E7
:1011A000C6F1A7C1C7F1A8C1C8F1A9C1C9F1AAC1B7
:1011B000CAF1ABC1CBF1ACC1CCF1ADC1CDF1AEC187
:1011C000CEF1AFC1CFF1B0C1D0F1B1C1D1F1B2C157
:1011D000D2F1B3C1D3F1B4C1D4F1B5C1D5F101019C
:1011E00055515B2756515C23E86A5D230E2E01EFB3
:1011F00009F05CC157F15DC158F15B6B5C6B5D6BD5
:10120000078E03EF09F002C0E0FF005001C0D8FFD5
:101210001000A6B209EF09F00CC0A9FF0BC0A8FF8F
:10122000A69EA69CA684F29E550EA76EAA0EA76E39
:10123000A682F28EA694A6B21BEF09F00C2A120029
:10124000A96EA69EA69CA680A8500C2A1200040196
:101250002C0E826F18EC0BF06EEC1CF00C5020EC96
:1012600009F0E8CF00F10C5020EC09F0E8CF01F1D3
:1012700001AF40EF09F00101FF0E026FFF0E036F97
:1012800011EC1CF029674CEF09F00401200E826F6D
:1012900018EC0BF051EF09F004012D0E826F18ECE1
:1012A0000BF03BEC1AF01200076A0F6A106A116A21
:1012B000126A0F010E0EC16E860EC06E030EC26E54
:1012C0000F01896A110E926E080E8A6EF10E936EEE
:1012D0008B6A980E946EF18EFC0E20EC09F0E8CF2C
:1012E0000BF00BA011800BA211820BA411840BA890
:1012F0001188C90E20EC09F0E8CF16F0CA0E20ECD8
:1013000009F0E8CF17F0CB0E20EC09F0E8CF18F089
:10131000196A1A6A0E6A01015B6B5C6B5D6B576B35
:10132000586BF29A0101476B486B496B4A6B4B6BE8
:101330004C6B4D6B4E6B4F6B506B516B526B456BE7
:10134000466BD76AD66A0F01280ED56EF28A9D9039
:10135000B00ECD6E01015E6B5F6B606B616B626B9B
:10136000636B646B656B666B676B686B696B536B08
:10137000546BCF6ACE6A0F9A0F9C0F9E9D80760E9B
:10138000CA6E9D8202013C0E006FCC6A160E20ECE4
:1013900009F0E8CF00F1170E20EC09F0E8CF01F1D9
:1013A000180E20EC09F0E8CF02F1190E20EC09F03C
:1013B000E8CF03F1010103AFF8EF09F06EEC1CF088
:1013C000160E0C6E00C10BF009EC09F0170E0C6E36
:1013D00001C10BF009EC09F0180E0C6E02C10BF004
:1013E00009EC09F0190E0C6E03C10BF009EC09F0C1
:1013F00000C18AF101C18BF102C18CF103C18DF1F1
:1014000000C18EF101C18FF102C190F103C191F1D0
:101410001A0E20EC09F0E8CF00F11B0E20EC09F0C9
:10142000E8CF01F11C0E20EC09F0E8CF02F11D0E0F
:1014300020EC09F0E8CF03F1010103AF4EEF0AF011
:101440006EEC1CF01A0E0C6E00C10BF009EC09F0EA
:101450001B0E0C6E01C10BF009EC09F01C0E0C6E9A
:1014600002C10BF009EC09F01D0E0C6E03C10BF06C
:1014700009EC09F01A0E20EC09F0E8CF00F11B0E80
:1014800020EC09F0E8CF01F11C0E20EC09F0E8CFC8
:1014900002F11D0E20EC09F0E8CF03F100C192F13A
:1014A00001C193F102C194F103C195F1240EAC6E18
:1014B000900EAB6E240EAC6E080EB86E000EB06EC1
:1014C0001F0EAF6E0401806B816B0F01900EAB6E2F
:1014D0000F019D8A0301806B816BC26B8B92136A33
:1014E000146A156A9D8607900001F28EF28C07B08F
:1014F000E8EF18F00FB041EF13F010BE41EF13F01A
:101500000301805181197F0BD8B4E8EF18F013EE76
:1015100000F081517F0BE126812BE7CFE8FFE00B44
:10152000D8B4E8EF18F023EE82F0C2513F0BD92671
:10153000E7CFDFFFC22BDF50780AD8A4E8EF18F01E
:1015400007808EC100F18FC101F190C102F191C1FC
:1015500003F10101040E046F000E056F000E066F0B
:10156000000E076F73EC1BF000AFC0EF0AF0010133
:10157000030E8E6F000E8F6F000E906F000E916F36
:1015800003018251720AD8B43EEF13F08251520A1D
:10159000D8B43EEF13F08251750AD8B43EEF13F081
:1015A0008251630AD8B4A2EF15F08251690AD8B407
:1015B000E5EF0FF082517A0AD8B4F8EF10F08251BB
:1015C000490AD8B484EF0FF08251500AD8B4A2EF80
:1015D0000EF08251700AD8B4E5EF0EF08251540A31
:1015E000D8B410EF0FF08251740AD8B456EF0FF050
:1015F0008251410AD8B42CEF0BF082516D0AD8B455
:10160000FAEF0DF082514D0AD8B413EF0EF082516B
:10161000730AD8B46EEF12F08251530AD8B4D3EFE4
:1016200012F08251590AD8B44BEF0DF0D9EF15F0F2
:10163000040114EE00F080517F0BE12682C4E7FF25
:10164000802B120004010D0E826F18EC0BF00A0EB5
:10165000826F18EC0BF012000401410E826F18EC3F
:101660000BF003018351310AD8B46BEF0CF0030186
:101670008351320AD8B4C1EF0BF003018351330A0E
:10168000D8B44AEF0BF004013F0E826F18EC0BF058
:10169000D7EF15F0CB0E20EC09F0E8CF0BF00401EA
:1016A0002C0E826F18EC0BF003018451450AD8B45C
:1016B0006EEF0BF003018451440AD8B471EF0BF0C4
:1016C00003018451300AD8B474EF0BF00301845144
:1016D000310AD8B478EF0BF083EF0BF00B9E7DEF5F
:1016E0000BF00B8E7DEF0BF0FC0E0B167DEF0BF06D
:1016F000FC0E0B160B807DEF0BF0CB0E0C6E0BC0AF
:101700000BF009EC09F00401330E826F18EC0BF0BA
:1017100004012C0E826F18EC0BF0CB0E20EC09F0BC
:10172000E8CF18F018BE9CEF0BF00401450E826F55
:1017300018EC0BF0A1EF0BF00401440E826F18ECD3
:101740000BF004012C0E826F18EC0BF00401300E2C
:10175000826F18EC0BF004012C0E826F18EC0BF06A
:1017600018B0BAEF0BF00401300E826F18EC0BF0DA
:10177000BFEF0BF00401310E826F18EC0BF0D7EFC6
:1017800015F0CA0E20EC09F0E8CF0BF004012C0E86
:10179000826F18EC0BF003018451450AD8B4F1EFC5
:1017A0000BF003018451440AD8B4F4EF0BF00301A9
:1017B00084514D0AD8B4FDEF0BF003018451410A66
:1017C000D8B4F7EF0BF003018451460AD8B4FAEF0E
:1017D0000BF003018451560AD8B405EF0CF016EF54
:1017E0000CF00B9E10EF0CF00B8E10EF0CF00B9C1E
:1017F00010EF0CF00B8C10EF0CF0F80E0B1685C3ED
:10180000E8FF070B0B1210EF0CF0C70E0B1685C389
:10181000E8FF070BE846E846E8460B1210EF0CF02D
:10182000CA0E0C6E0BC00BF009EC09F0CA0E20ECCE
:1018300009F0E8CF17F00401320E826F18EC0BF0BC
:1018400004012C0E826F18EC0BF017BE2FEF0CF07A
:101850000401450E826F18EC0BF034EF0CF004011C
:10186000440E826F18EC0BF004012C0E826F18EC02
:101870000BF017C0E8FF070BE8CF82F40401300E2D
:10188000822718EC0BF004012C0E826F18EC0BF081
:1018900017BC52EF0CF00401410E826F18EC0BF0F4
:1018A00057EF0CF00401460E826F18EC0BF00401A8
:1018B0002C0E826F18EC0BF017C0E8FF380BE842D3
:1018C000E842E842E8CF82F40401300E822718ECA7
:1018D0000BF0D7EF15F0C90E20EC09F0E8CF0BF0B4
:1018E00004012C0E826F18EC0BF003018451450AA1
:1018F000D8B489EF0CF003018451440AD8B48CEFBA
:101900000CF0030184514D0AD8B48FEF0CF09DEF19
:101910000CF00B9E97EF0CF00B8E97EF0CF0F80E7F
:101920000B1685C3E8FF070B0B1297EF0CF0C90EDF
:101930000C6E0BC00BF009EC09F00401310E826F44
:1019400018EC0BF004012C0E826F18EC0BF0C90E92
:1019500020EC09F0E8CF16F016BE06D00401450EC3
:10196000826F18EC0BF005D00401440E826F18EC66
:101970000BF004012C0E826F18EC0BF016C0E8FF80
:10198000070BE8CF82F40401300E822718EC0BF02D
:1019900004012C0E826F18EC0BF007806EEC1CF02B
:1019A00025C0E8FF003B00430043030B11EC1CF093
:1019B00033C182F40401300E822718EC0BF00401CD
:1019C0002C0E826F18EC0BF06EEC1CF025C001F1B0
:1019D000019F019D26C000F1010111EC1CF02FC1F7
:1019E00082F40401300E822718EC0BF030C182F42F
:1019F0000401300E822718EC0BF031C182F404018F
:101A0000300E822718EC0BF032C182F40401300E44
:101A1000822718EC0BF033C182F40401300E8227C8
:101A200018EC0BF004012C0E826F18EC0BF06EEC2E
:101A30001CF027C001F128C000F1D8900133003319
:101A4000D89001330033010111EC1CF02FC182F456
:101A50000401300E822718EC0BF030C182F404012F
:101A6000300E822718EC0BF031C182F40401300EE5
:101A7000822718EC0BF032C182F40401300E822769
:101A800018EC0BF033C182F40401300E822718ECFD
:101A90000BF0D7EF15F0FC0E20EC09F0E8CF0BF0BF
:101AA00003018351520AD8B482EF0DF00301835130
:101AB000720AD8B485EF0DF003018351500AD8B4EF
:101AC00088EF0DF003018351700AD8B48BEF0DF04D
:101AD00003018351550AD8B48EEF0DF003018351F1
:101AE000750AD8B491EF0DF003018351430AD8B4BD
:101AF0009AEF0DF003018351630AD8B49DEF0DF006
:101B0000A6EF0DF00B90A0EF0DF00B80A0EF0DF005
:101B10000B92A0EF0DF00B82A0EF0DF00B94A0EF55
:101B20000DF00B84A0EF0DF00B96A0EF0DF00B86DF
:101B3000A0EF0DF00B98A0EF0DF00B88A0EF0DF0CB
:101B4000FC0E0C6E0BC00BF009EC09F00401590EF1
:101B5000826F18EC0BF01190119211941198FC0EF9
:101B600020EC09F0E8CF0BF00BA011800BA2118242
:101B70000BA411840BA8118811A0C6EF0DF004016D
:101B8000520E826F18EC0BF0CBEF0DF00401720EC9
:101B9000826F18EC0BF011A8D5EF0DF00401430E85
:101BA000826F18EC0BF0DAEF0DF00401630E826F18
:101BB00018EC0BF011A2E4EF0DF00401500E826F4F
:101BC00018EC0BF0E9EF0DF00401700E826F18ECC9
:101BD0000BF011A4F3EF0DF00401550E826F18EC19
:101BE0000BF0F8EF0DF00401750E826F18EC0BF09E
:101BF000D7EF15F004016D0E826F18EC0BF00301A6
:101C00008351300AD8B452EF0EF003018351310AE8
:101C1000D8B465EF0EF003018351320AD8B478EFDF
:101C20000EF0D9EF15F004014D0E826F18EC0BF099
:101C3000AFEC1CF084C331F185C332F186C333F1BC
:101C40000101296BBCEC1CF033EC1CF00301835147
:101C5000300AD8B43AEF0EF003018351310AD8B4F8
:101C600042EF0EF003018351320AD8B44AEF0EF06E
:101C7000D9EF15F0FD0E0C6E00C10BF009EC09F068
:101C800052EF0EF0FE0E0C6E00C10BF009EC09F0E5
:101C900065EF0EF0FF0E0C6E00C10BF009EC09F0C1
:101CA00078EF0EF00401300E826F18EC0BF0040197
:101CB0002C0E826F18EC0BF06EEC1CF0FD0E20EC7D
:101CC00009F0E8CF00F189EF0EF00401310E826FC8
:101CD00018EC0BF004012C0E826F18EC0BF06EEC7C
:101CE0001CF0FE0E20EC09F0E8CF00F189EF0EF0B9
:101CF0000401320E826F18EC0BF06EEC1CF0040144
:101D00002C0E826F18EC0BF0FF0E20EC09F0E8CFE0
:101D100000F111EC1CF031C182F40401300E822775
:101D200018EC0BF032C182F40401300E822718EC5B
:101D30000BF033C182F40401300E822718EC0BF053
:101D4000D7EF15F083C32AF184C32BF185C32CF19F
:101D500086C32DF187C32EF188C32FF189C330F1DB
:101D60008AC331F18BC332F18CC333F10101BCEC76
:101D70001CF033EC1CF0160E0C6E00C10BF009ECDD
:101D800009F0170E0C6E01C10BF009EC09F0180EEA
:101D90000C6E02C10BF009EC09F0190E0C6E03C1B8
:101DA0000BF009EC09F000C18AF101C18BF102C10D
:101DB0008CF103C18DF100C18EF101C18FF102C11F
:101DC00090F103C191F184EF0FF083C32AF184C332
:101DD0002BF185C32CF186C32DF187C32EF188C367
:101DE0002FF189C330F18AC331F18BC332F18CC337
:101DF00033F10101BCEC1CF033EC1CF000C18AF1A2
:101E000001C18BF102C18CF103C18DF100C18EF1D2
:101E100001C18FF102C190F103C191F184EF0FF084
:101E200083C32AF184C32BF185C32CF186C32DF122
:101E300087C32EF188C32FF189C330F18AC331F1F2
:101E40008CC332F18DC333F10101BCEC1CF033ECD7
:101E50001CF00101000E046F000E056F010E066FED
:101E6000000E076F84EC1BF01A0E0C6E00C10BF015
:101E700009EC09F01B0E0C6E01C10BF009EC09F026
:101E80001C0E0C6E02C10BF009EC09F01D0E0C6E5D
:101E900003C10BF009EC09F000C192F101C193F10B
:101EA00002C194F103C195F184EF0FF083C32AF1CD
:101EB00084C32BF185C32CF186C32DF187C32EF18A
:101EC00088C32FF189C330F18AC331F18CC332F159
:101ED0008DC333F10101BCEC1CF033EC1CF00101AB
:101EE000000E046F000E056F010E066F000E076FE7
:101EF00084EC1BF000C192F101C193F102C194F195
:101F000003C195F184EF0FF0160E20EC09F0E8CF35
:101F100000F1170E20EC09F0E8CF01F1180E20ECCB
:101F200009F0E8CF02F1190E20EC09F0E8CF03F137
:101F300011EC1CF0F4EC19F00401730E826F18EC34
:101F40000BF004012C0E826F18EC0BF08AC100F12B
:101F50008BC101F18CC102F18DC103F111EC1CF0B8
:101F6000F4EC19F00401730E826F18EC0BF004010D
:101F70002C0E826F18EC0BF01A0E20EC09F0E8CF53
:101F800000F11B0E20EC09F0E8CF01F11C0E20EC53
:101F900009F0E8CF02F11D0E20EC09F0E8CF03F1C3
:101FA000F4EC15F004012C0E826F18EC0BF092C1CA
:101FB00000F193C101F194C102F195C103F1F4EC78
:101FC00015F022EC0BF0D9EF15F00401690E826FC9
:101FD00018EC0BF004012C0E826F18EC0BF00101D1
:101FE000040E006F000E016F000E026F000E036FF3
:101FF00011EC1CF02CC182F40401300E822718EC85
:102000000BF02DC182F40401300E822718EC0BF086
:102010002EC182F40401300E822718EC0BF02FC180
:1020200082F40401300E822718EC0BF030C182F4E8
:102030000401300E822718EC0BF031C182F4040148
:10204000300E822718EC0BF032C182F40401300EFE
:10205000822718EC0BF033C182F40401300E822782
:1020600018EC0BF004012C0E826F18EC0BF0010140
:10207000030E006F000E016F000E026F000E036F63
:1020800011EC1CF02CC182F40401300E822718ECF4
:102090000BF02DC182F40401300E822718EC0BF0F6
:1020A0002EC182F40401300E822718EC0BF02FC1F0
:1020B00082F40401300E822718EC0BF030C182F458
:1020C0000401300E822718EC0BF031C182F40401B8
:1020D000300E822718EC0BF032C182F40401300E6E
:1020E000822718EC0BF033C182F40401300E8227F2
:1020F00018EC0BF004012C0E826F18EC0BF00101B0
:10210000290E006F000E016F000E026F000E036FAC
:1021100011EC1CF02CC182F40401300E822718EC63
:102120000BF02DC182F40401300E822718EC0BF065
:102130002EC182F40401300E822718EC0BF02FC15F
:1021400082F40401300E822718EC0BF030C182F4C7
:102150000401300E822718EC0BF031C182F4040127
:10216000300E822718EC0BF032C182F40401300EDD
:10217000822718EC0BF033C182F40401300E822761
:1021800018EC0BF004012C0E826F18EC0BF0200EF3
:10219000F86EF76AF66A04010900F5CF82F418ECCC
:1021A0000BF00900F5CF82F418EC0BF00900F5CF25
:1021B00082F418EC0BF00900F5CF82F418EC0BF068
:1021C0000900F5CF82F418EC0BF00900F5CF82F48A
:1021D00018EC0BF00900F5CF82F418EC0BF00900B5
:1021E000F5CF82F418EC0BF022EC0BF0D9EF15F0E0
:1021F0008351630AD8A4D9EF15F08451610AD8A499
:10220000D9EF15F085516C0AD8A4D9EF15F0865195
:10221000410A42E08651440A1BE08651420AD8B482
:102220005FEF11F08651350AD8B463EF17F086518D
:10223000360AD8B4B8EF17F08651370AD8B421EF70
:1022400018F08651380AD8B47FEF18F0D9EF15F09E
:102250000798079A04017A0E826F18EC0BF00401BC
:10226000780E826F18EC0BF00401640E826F18EC8C
:102270000BF081A843EF11F00401550E826F18ECAA
:102280000BF048EF11F004014C0E826F18EC0BF0CC
:1022900022EC0BF0D9EF15F00788079A04017A0EAB
:1022A000826F18EC0BF00401410E826F18EC0BF0FA
:1022B0000401610E826F18EC0BF039EF11F00798F2
:1022C000078A04017A0E826F18EC0BF00401420EAB
:1022D000826F18EC0BF00401610E826F18EC0BF0AA
:1022E00039EF11F0010166677DEF11F067677DEF4F
:1022F00011F068677DEF11F0696795EF11F04F6796
:1023000089EF11F0506789EF11F0516789EF11F0F3
:10231000526795EF11F00101000E006F000E016F82
:10232000000E026F000E036F120011B8A3EF11F040
:102330000101620E046F010E056F000E066F000EA4
:10234000076FACEF11F00101A70E046F020E056FCD
:10235000000E066F000E076F66C100F167C101F144
:1023600068C102F169C103F173EC1BF003BF2AEFEE
:1023700012F0119A0101000E046FA80E056F550EA0
:10238000066F020E076F66C100F167C101F168C1F7
:1023900002F169C103F166C186F167C187F168C1C5
:1023A00088F169C189F173EC1BF003BFE3EF11F011
:1023B0000101000E866FA80E876F550E886F020E02
:1023C000896F118A119C0E0E20EC09F0E8CF18F1EC
:1023D0000F0E20EC09F0E8CF19F1100E20EC09F0F7
:1023E000E8CF1AF1110E20EC09F0E8CF1BF1BCEC9C
:1023F0001AF086C104F187C105F188C106F189C1CF
:1024000007F173EC1BF0078280EC1AF0BCEC1AF0B9
:10241000079280EC1AF086C100F187C101F188C1F2
:1024200002F189C103F1079280EC1AF0CC0E046F1F
:10243000E00E056F870E066F050E076F73EC1BF03D
:1024400000C118F101C119F102C11AF103C11BF158
:1024500065EF12F0119C0101800E006F1A0E016FE2
:10246000060E026F000E036F4FC104F150C105F15B
:1024700051C106F152C107F173EC1BF003AF46EFF7
:1024800012F06EEC1CF0118C119A12000E0E20EC62
:1024900009F0E8CF18F10F0E20EC09F0E8CF19F1A0
:1024A000100E20EC09F0E8CF1AF1110E20EC09F023
:1024B000E8CF1BF14FC100F150C101F151C102F150
:1024C00052C103F1078280EC1AF018C100F119C162
:1024D00001F11AC102F11BC103F112000401730ED4
:1024E000826F18EC0BF004012C0E826F18EC0BF0CD
:1024F000078462C166F163C167F164C168F165C1B7
:1025000069F14BC14FF14CC150F14DC151F14EC178
:1025100052F157C159F158C15AF1079494EC12F095
:1025200022EC0BF0D9EF15F066C100F167C101F1A3
:1025300068C102F169C103F1010111EC1CF0F4EC76
:1025400019F00401630E826F18EC0BF004012C0EDD
:10255000826F18EC0BF04FC100F150C101F151C175
:1025600002F152C103F1010111EC1CF0F4EC19F07D
:102570000401660E826F18EC0BF004012C0E826FC2
:1025800018EC0BF06EEC1CF059C100F15AC101F1CE
:10259000010111EC1CF0F4EC19F00401740E826FCF
:1025A00018EC0BF0120010820401530E826F18EC2D
:1025B0000BF004012C0E826F18EC0BF083C32AF190
:1025C00084C32BF185C32CF186C32DF187C32EF173
:1025D00088C32FF189C330F18AC331F18BC332F143
:1025E0008CC333F10101BCEC1CF033EC1CF000C1D6
:1025F00066F101C167F102C168F103C169F18EC3DF
:102600002AF18FC32BF190C32CF191C32DF192C30A
:102610002EF193C32FF194C330F195C331F196C3DA
:1026200032F197C333F10101BCEC1CF033EC1CF028
:1026300000C14FF101C150F102C151F103C152F18A
:10264000AFEC1CF099C32FF19AC330F19BC331F169
:102650009CC332F19DC333F10101BCEC1CF033EC9F
:102660001CF000C159F101C15AF194EC12F00401BF
:102670002C0E826F18EC0BF048EF13F018A001D06D
:10268000108C8251520A03E10F8248EF13F00F922F
:102690008251750A03E110844FEF13F0109411A0DA
:1026A00056EF13F011A456EF13F010848251550A1F
:1026B00003E110865DEF13F01096078410B2BAEFB5
:1026C00013F010A4A6EF13F0B6C166F1B7C167F11D
:1026D000B8C168F1B9C169F1BAC16AF1BBC16BF1A6
:1026E000BCC16CF1BDC16DF1BEC16EF1BFC16FF176
:1026F000C0C170F1C1C171F1C2C172F1C3C173F146
:10270000C4C174F1C5C175F1C6C176F1C7C177F115
:10271000C8C178F1C9C179F1CAC17AF1CBC17BF1E5
:10272000CCC17CF1CDC17DF1CEC17EF1CFC17FF1B5
:10273000D0C180F1D1C181F1D2C182F1D3C183F185
:10274000D4C184F1D5C185F1AEEF13F062C166F159
:1027500063C167F164C168F165C169F14BC14FF1B3
:102760004CC150F14DC151F14EC152F157C159F117
:1027700058C15AF107940FA0DCEF13F001019267E2
:10278000C9EF13F09367C9EF13F09467C9EF13F023
:102790009567CDEF13F0DCEF13F072EC11F092C1FE
:1027A00004F193C105F194C106F195C107F173ECF1
:1027B0001BF003BF9FEF15F072EC11F00101000E4A
:1027C000046F000E056F010E066F000E076FA4EC7C
:1027D0001BF011A01BEF14F011A21BEF14F011EC71
:1027E0001CF02967F6EF13F0FDEF13F004012D0E36
:1027F000826F18EC0BF09DEF15F030C182F40401EC
:10280000300E822718EC0BF031C182F40401300E37
:10281000822718EC0BF032C182F40401300E8227BB
:1028200018EC0BF033C182F40401300E822718EC4F
:102830000BF09DEF15F010AE4BD0109E00C108F1CB
:1028400001C109F102C10AF103C10BF111EC1CF045
:1028500030C1D6F131C1D7F132C1D8F133C1D9F18C
:1028600008C100F109C101F10AC102F10BC103F174
:1028700001016C0E046F070E056F000E066F000E4F
:10288000076F73EC1BF003BF04D00101550EDA6F24
:102890001CD008C100F109C101F10AC102F10BC14C
:1028A00003F10101A40E046F060E056F000E066F02
:1028B000000E076F73EC1BF003BF04D001017F0E05
:1028C000DA6F03D00101FF0EDA6F198E9FEF15F05A
:1028D00010A472EF14F00401750E826F18EC0BF067
:1028E00077EF14F00401720E826F18EC0BF0040104
:1028F0002C0E826F18EC0BF011EC1CF0296786EFA0
:1029000014F00401200E826F89EF14F004012D0EE3
:10291000826F18EC0BF030C182F40401300E822774
:1029200018EC0BF031C182F40401300E822718EC50
:102930000BF004012E0E826F18EC0BF032C182F402
:102940000401300E822718EC0BF033C182F404012D
:10295000300E822718EC0BF004016D0E826F18EC1C
:102960000BF004012C0E826F18EC0BF04FC100F13C
:1029700050C101F151C102F152C103F1010111EC49
:102980001CF0F4EC19F00401480E826F18EC0BF007
:1029900004017A0E826F18EC0BF004012C0E826F8A
:1029A00018EC0BF066C100F167C101F168C102F1DA
:1029B00069C103F1010111EC1CF0F4EC19F0040100
:1029C000630E826F18EC0BF004012C0E826F18EC72
:1029D0000BF066C100F167C101F168C102F169C184
:1029E00003F101010A0E046F000E056F000E066F61
:1029F000000E076F84EC1BF0000E046F120E056FC3
:102A0000000E066F000E076FA4EC1BF011EC1CF01B
:102A10002AC182F40401300E822718EC0BF02BC17E
:102A200082F40401300E822718EC0BF02CC182F4E2
:102A30000401300E822718EC0BF02DC182F4040142
:102A4000300E822718EC0BF02EC182F40401300EF8
:102A5000822718EC0BF02FC182F40401300E82277C
:102A600018EC0BF030C182F40401300E822718EC10
:102A70000BF004012E0E826F18EC0BF031C182F4C2
:102A80000401300E822718EC0BF032C182F40401ED
:102A9000300E822718EC0BF033C182F40401300EA3
:102AA000822718EC0BF00401730E826F18EC0BF008
:102AB00004012C0E826F18EC0BF06EEC1CF059C167
:102AC00000F15AC101F103EC17F00FB26BEF15F0F2
:102AD0000FA09DEF15F004012C0E826F18EC0BF087
:102AE000200EF86EF76AF66A04010900F5CF82F449
:102AF00018EC0BF00900F5CF82F418EC0BF009008C
:102B0000F5CF82F418EC0BF00900F5CF82F418EC45
:102B10000BF00900F5CF82F418EC0BF00900F5CFAB
:102B200082F418EC0BF00900F5CF82F418EC0BF0EE
:102B30000900F5CF82F418EC0BF022EC0BF00F90AB
:102B4000D9EF15F00401630E826F18EC0BF004014D
:102B50002C0E826F18EC0BF0DFEC15F004012C0E3C
:102B6000826F18EC0BF052EC16F004012C0E826F01
:102B700018EC0BF0CEEC16F004012C0E826F18EC62
:102B80000BF00101F80E006FCD0E016F660E026FA3
:102B9000030E036FF4EC15F004012C0E826F18EC99
:102BA0000BF0E4EC16F022EC0BF0D9EF15F022EC70
:102BB0000BF00301C26B07901092E8EF18F0D89069
:102BC0000E0E20EC09F0E8CF00F10F0E20EC09F01A
:102BD000E8CF01F1100E20EC09F0E8CF02F1110E60
:102BE00020EC09F0E8CF03F10101000E046F000EA4
:102BF000056F010E066F000E076FA4EC1BF011ECC1
:102C00001CF02AC182F40401300E822718EC0BF06C
:102C10002BC182F40401300E822718EC0BF02CC17A
:102C200082F40401300E822718EC0BF02DC182F4DF
:102C30000401300E822718EC0BF02EC182F404013F
:102C4000300E822718EC0BF02FC182F40401300EF5
:102C5000822718EC0BF030C182F40401300E822779
:102C600018EC0BF031C182F40401300E822718EC0D
:102C70000BF004012E0E826F18EC0BF032C182F4BF
:102C80000401300E822718EC0BF033C182F40401EA
:102C9000300E822718EC0BF004016D0E826F18ECD9
:102CA0000BF01200120E20EC09F0E8CF00F1130E29
:102CB00020EC09F0E8CF01F1140E20EC09F0E8CF88
:102CC00002F1150E20EC09F0E8CF03F101010A0E24
:102CD000046F000E056F000E066F000E076F84EC88
:102CE0001BF0000E046F120E056F000E066F000E33
:102CF000076FA4EC1BF011EC1CF02AC182F4040154
:102D0000300E822718EC0BF02BC182F40401300E38
:102D1000822718EC0BF02CC182F40401300E8227BC
:102D200018EC0BF02DC182F40401300E822718EC50
:102D30000BF02EC182F40401300E822718EC0BF048
:102D40002FC182F40401300E822718EC0BF030C141
:102D500082F40401300E822718EC0BF004012E0ED1
:102D6000826F18EC0BF031C182F40401300E82271F
:102D700018EC0BF032C182F40401300E822718ECFB
:102D80000BF033C182F40401300E822718EC0BF0F3
:102D90000401730E826F18EC0BF012000A0E20EC87
:102DA00009F0E8CF00F10B0E20EC09F0E8CF01F1BB
:102DB0000C0E20EC09F0E8CF02F10D0E20EC09F02A
:102DC000E8CF03F103EF17F0060E20EC09F0E8CF8F
:102DD00000F1070E20EC09F0E8CF01F1080E20EC1D
:102DE00009F0E8CF02F1090E20EC09F0E8CF03F179
:102DF00003EF17F001016EEC1CF0078457C100F1DE
:102E000058C101F107940101E80E046F800E056FAF
:102E1000000E066F000E076F84EC1BF0000E046FAF
:102E2000040E056F000E066F000E076FA4EC1BF07A
:102E3000880E046F130E056F000E066F000E076FED
:102E400073EC1BF00A0E046F000E056F000E066F88
:102E5000000E076FA4EC1BF011EC1CF001012967B8
:102E600037EF17F00401200E826F3AEF17F00401DC
:102E70002D0E826F18EC0BF030C182F40401300E7D
:102E8000822718EC0BF031C182F40401300E822746
:102E900018EC0BF032C182F40401300E822718ECDA
:102EA0000BF004012E0E826F18EC0BF033C182F48C
:102EB0000401300E822718EC0BF00401430E826FE0
:102EC00018EC0BF0120087C32AF188C32BF189C3D9
:102ED0002CF18AC32DF18BC32EF18CC32FF18DC33E
:102EE00030F18EC331F190C332F191C333F101015E
:102EF000296BBCEC1CF033EC1CF00101000E046FDC
:102F0000000E056F010E066F000E076F84EC1BF0BC
:102F10000E0E0C6E00C10BF009EC09F00F0E0C6EDA
:102F200001C10BF009EC09F0100E0C6E02C10BF0A0
:102F300009EC09F0110E0C6E03C10BF009EC09F05D
:102F400004017A0E826F18EC0BF004012C0E826FD4
:102F500018EC0BF00401350E826F18EC0BF0040135
:102F60002C0E826F18EC0BF0DFEC15F048EF11F02F
:102F700087C32AF188C32BF189C32CF18AC32DF1B1
:102F80008BC32EF18CC32FF18DC330F18EC331F181
:102F900090C332F191C333F10101296BBCEC1CF0F9
:102FA00033EC1CF0880E046F130E056F000E066FD5
:102FB000000E076F78EC1BF0000E046F040E056F17
:102FC000000E066F000E076F84EC1BF00101E80E87
:102FD000046F800E056F000E066F000E076FA4ECE5
:102FE0001BF00A0E0C6E00C10BF009EC09F00B0E81
:102FF0000C6E01C10BF009EC09F00C0E0C6E02C155
:103000000BF009EC09F00D0E0C6E03C10BF009EC8E
:1030100009F004017A0E826F18EC0BF004012C0EFB
:10302000826F18EC0BF00401360E826F18EC0BF077
:1030300004012C0E826F18EC0BF0CEEC16F048EF6A
:1030400011F087C32AF188C32BF189C32CF18AC3FD
:103050002DF18BC32EF18CC32FF18DC330F18FC3B3
:1030600031F190C332F191C333F10101BCEC1CF09A
:1030700033EC1CF0000E046F120E056F000E066F8D
:10308000000E076F84EC1BF001010A0E046F000EA6
:10309000056F000E066F000E076FA4EC1BF0120EFA
:1030A0000C6E00C10BF009EC09F0130E0C6E01C19F
:1030B0000BF009EC09F0140E0C6E02C10BF009ECD8
:1030C00009F0150E0C6E03C10BF009EC09F00401B8
:1030D0007A0E826F18EC0BF004012C0E826F18EC44
:1030E0000BF00401370E826F18EC0BF004012C0E6C
:1030F000826F18EC0BF052EC16F048EF11F087C31A
:103100002AF188C32BF189C32CF18AC32DF18BC31B
:103110002EF18CC32FF18DC330F18EC331F190C3EA
:1031200032F191C333F10101296BBCEC1CF033EC9B
:103130001CF0880E046F130E056F000E066F000E54
:10314000076F78EC1BF0000E046F040E056F000E85
:10315000066F000E076F84EC1BF00101E80E046F90
:10316000800E056F000E066F000E076FA4EC1BF0BB
:10317000060E0C6E00C10BF009EC09F0070E0C6E88
:1031800001C10BF009EC09F0080E0C6E02C10BF046
:1031900009EC09F0090E0C6E03C10BF009EC09F003
:1031A00004017A0E826F18EC0BF004012C0E826F72
:1031B00018EC0BF00401380E826F18EC0BF00401D0
:1031C0002C0E826F18EC0BF0E4EC16F048EF11F0C7
:1031D00081A8A6EF19F007A85FEF19F00101800E92
:1031E000006F1A0E016F060E026F000E036F4BC1C7
:1031F00004F14CC105F14DC106F14EC107F173EC6C
:103200001BF003BFA6EF19F0EEEC19F04BC100F173
:103210004CC101F14DC102F14EC103F1078280ECB6
:103220001AF018C104F119C105F11AC106F11BC148
:1032300007F1F80E006FCD0E016F660E026F030EE0
:10324000036F73EC1BF00E0E0C6E00C10BF009EC5B
:1032500009F00F0E0C6E01C10BF009EC09F0100E15
:103260000C6E02C10BF009EC09F0110E0C6E03C1DB
:103270000BF009EC09F0078401016EEC1CF057C15A
:1032800000F158C101F107940A0E0C6E00C10BF059
:1032900009EC09F00B0E0C6E01C10BF009EC09F002
:1032A0000C0E0C6E02C10BF009EC09F00D0E0C6E49
:1032B00003C10BF009EC09F00798A6EF19F007AA73
:1032C000A6EF19F0078401016EEC1CF057C100F164
:1032D00058C101F10794060E0C6E00C10BF009EC09
:1032E00009F0070E0C6E01C10BF009EC09F0080E95
:1032F0000C6E02C10BF009EC09F0090E0C6E03C153
:103300000BF009EC09F0078462C100F163C101F11F
:1033100064C102F165C103F10794120E0C6E00C185
:103320000BF009EC09F0130E0C6E01C10BF009EC67
:1033300009F0140E0C6E02C10BF009EC09F0150E29
:103340000C6E03C10BF009EC09F0079A04018051DF
:1033500081197F0B0BE09EA809D014EE00F081517B
:103360007F0BE126E750812B0F01AD6E77EF0AF05E
:1033700018C100F119C101F11AC102F11BC103F119
:10338000000E046F000E056F010E066F000E076F32
:10339000A4EC1BF029A1E3EF19F02051D8B4E3EF1E
:1033A00019F018C100F119C101F11AC102F11BC1D4
:1033B00003F1000E046F000E056F0A0E066F000E7B
:1033C000076FA4EC1BF0120001010451001305511A
:1033D0000113065102130751031312000101186B68
:1033E000196B1A6B1B6B12002AC182F40401300E98
:1033F000822718EC0BF02BC182F40401300E8227D7
:1034000018EC0BF02CC182F40401300E822718EC6A
:103410000BF02DC182F40401300E822718EC0BF062
:103420002EC182F40401300E822718EC0BF02FC15C
:1034300082F40401300E822718EC0BF030C182F4C4
:103440000401300E822718EC0BF031C182F4040124
:10345000300E822718EC0BF032C182F40401300EDA
:10346000822718EC0BF033C182F40401300E82275E
:1034700018EC0BF012002FC182F40401300E8227E9
:1034800018EC0BF030C182F40401300E822718ECE6
:103490000BF031C182F40401300E822718EC0BF0DE
:1034A00032C182F40401300E822718EC0BF033C1D4
:1034B00082F40401300E822718EC0BF01200060E85
:1034C0001B6E060E1C6E060E1D6E1B2E65EF1AF08F
:1034D0001C2E65EF1AF01D2E65EF1AF08B84020E7C
:1034E0001B6E020E1C6E020E1D6E1B2E75EF1AF067
:1034F0001C2E75EF1AF01D2E75EF1AF08B9412002A
:103500000101005305E1015303E1025301E1002BE6
:1035100043EC1BF06EEC1CF03951006F3A51016F17
:10352000420E046F4B0E056F000E066F000E076F04
:1035300084EC1BF000C104F101C105F102C106F1E8
:1035400003C107F118C100F119C101F11AC102F15B
:103550001BC103F107B2B1EF1AF078EC1BF0B3EF27
:103560001AF073EC1BF000C118F101C119F102C18E
:103570001AF103C11BF112006EEC1CF059C100F1ED
:103580005AC101F1060E20EC09F0E8CF04F1070E54
:1035900020EC09F0E8CF05F1080E20EC09F0E8CFA7
:1035A00006F1090E20EC09F0E8CF07F173EC1BF0EF
:1035B00000C124F101C125F102C126F103C127F1A7
:1035C000290E046F000E056F000E066F000E076FC8
:1035D00084EC1BF0EE0E046F430E056F000E066FB9
:1035E000000E076F78EC1BF024C104F125C105F132
:1035F00026C106F127C107F184EC1BF000C11CF1C4
:1036000001C11DF102C11EF103C11FF1120E20EC18
:1036100009F0E8CF04F1130E20EC09F0E8CF05F132
:10362000140E20EC09F0E8CF06F1150E20EC09F09D
:10363000E8CF07F10D0E006F000E016F000E026F54
:10364000000E036F84EC1BF0180E046F000E056F64
:10365000000E066F000E076FA4EC1BF01CC104F1F6
:103660001DC105F11EC106F11FC107F178EC1BF069
:103670006A0E046F2A0E056F000E066F000E076FAC
:1036800073EC1BF01200BF0EFA6E200E3A6F396B0E
:10369000D8900037013702370337D8B054EF1BF00A
:1036A0003A2F49EF1BF039073A070353D8B41200F9
:1036B0000331070B80093F6F03390F0B010F396F7F
:1036C00080EC5FF0406F390580EC5FF0405D405F5B
:1036D000396B3F33D8B0392739333FA969EF1BF035
:1036E000405139271200010193EC1CF0D8B01200B0
:1036F000010103510719346F56EC1CF0D8900751A3
:10370000031934AF800F12000101346B7AEC1CF006
:10371000D8A090EC1CF0D8B0120065EC1CF06EEC58
:103720001CF01F0E366FA6EC1CF00B35D8B056EC13
:103730001CF0D8A00335D8B01200362F93EF1BF041
:1037400034B17DEC1CF012000101346B0451051101
:10375000061107110008D8A07AEC1CF0D8A090EC54
:103760001CF0D8B01200086B096B0A6B0B6BA6EC4F
:103770001CF01F0E366FA6EC1CF007510B5DD8A491
:10378000CEEF1BF006510A5DD8A4CEEF1BF0055119
:10379000095DD8A4CEEF1BF00451085DD8A0E1EF7D
:1037A0001BF00451085F0551D8A0053D095F065183
:1037B000D8A0063D0A5F0751D8A0073D0B5FD890FF
:1037C0000081362FBBEF1BF034B17DEC1CF0346B65
:1037D0007AEC1CF0D890AAEC1CF007510B5DD8A431
:1037E000FEEF1BF006510A5DD8A4FEEF1BF0055159
:1037F000095DD8A4FEEF1BF00451085DD8A00DEFC1
:103800001CF0003F0DEF1CF0013F0DEF1CF0023FDC
:103810000DEF1CF0032BD8B4120034B17DEC1CF07A
:1038200012000101346B7AEC1CF0D8B01200AFEC3E
:103830001CF0200E366F003701370237033711EEC8
:1038400033F00A0E376FE7360A0EE75CD8B0E76E42
:10385000E552372F23EF1CF0362F1BEF1CF034B14D
:103860002981D890120001010A0E346F200E366FA4
:1038700011EE29F03451376F0A0ED890E652D8B0C5
:10388000E726E732372F3EEF1CF0033302330133D4
:103890000033362F38EF1CF0E750FF0FD8A0033568
:1038A000D8B0120029B17DEC1CF0120004510027A1
:1038B0000551D8B0053D01270651D8B0063D022775
:1038C0000751D8B0073D032712000051086F01517E
:1038D000096F02510A6F03510B6F12000101006B57
:1038E000016B026B036B12000101046B056B066B2D
:1038F000076B12000335D8A012000351800B001F84
:10390000011F021F031F003F8DEF1CF0013F8DEFD1
:103910001CF0023F8DEF1CF0032B342B032512000B
:103920000735D8A012000751800B041F051F061F82
:10393000071F043FA3EF1CF0053FA3EF1CF0063F59
:10394000A3EF1CF0072B342B07251200003701379B
:1039500002370337083709370A370B3712000101DE
:10396000296B2A6B2B6B2C6B2D6B2E6B2F6B306B9B
:10397000316B326B336B120001012A510F0B2A6F2E
:103980002B510F0B2B6F2C510F0B2C6F2D510F0B3D
:103990002D6F2E510F0B2E6F2F510F0B2F6F30519C
:1039A0000F0B306F31510F0B316F32510F0B326FE4
:1039B00033510F0B336F120000011550FF0A01E164
:1039C0001200390EC86E800EC76E280EC66E000E2D
:1039D000C56E1450000AD8B417EF1DF01450010A38
:1039E000D8B430EF1DF01450020AD8B449EF1DF0DE
:1039F0001450030AD8B462EF1DF01450040AD8B46E
:103A00008AEF1DF01450050AD8B4A3EF1DF014502E
:103A1000060AD8B4BCEF1DF01450070AD8B4D5EF8D
:103A20001DF01450080AD8B4EEEF1DF01200155026
:103A3000000AD8B40DEF1EF01550010AD8B411EFEA
:103A40001EF01550020AD8B415EF1EF01550030AE7
:103A5000D8B419EF1EF01550040AD8B488EF1EF040
:103A60001550000AD8B41DEF1EF01550010AD8B445
:103A700021EF1EF01550020AD8B425EF1EF01550A4
:103A8000030AD8B429EF1EF01550040AD8B488EF01
:103A90001EF01550000AD8B42DEF1EF01550010A83
:103AA000D8B431EF1EF01550020AD8B435EF1EF02D
:103AB0001550030AD8B439EF1EF01550040AD8B4D3
:103AC00088EF1EF01550000AD8B446EF1EF01550CE
:103AD000010AD8B44AEF1EF01550020AD8B44EEFCE
:103AE0001EF01550030AD8B462EF1EF01550040AF8
:103AF000D8B466EF1EF01550050AD8B46AEF1EF070
:103B00001550060AD8B46EEF1EF01550070AD8B447
:103B100071EF1EF01550000AD8B475EF1EF0155065
:103B2000010AD8B479EF1EF01550020AD8B47DEF1F
:103B30001EF01550030AD8B481EF1EF01550040A88
:103B4000D8B484EF1EF01550000AD8B48CEF1EF0E4
:103B50001550010AD8B490EF1EF01550020AD8B4DF
:103B600094EF1EF01550030AD8B498EF1EF01550CC
:103B7000040AD8B488EF1EF01550000AD8B4A2EF9A
:103B80001EF01550010AD8B4A6EF1EF01550020A17
:103B9000D8B4AAEF1EF01550030AD8B4AEEF1EF049
:103BA0001550040AD8B488EF1EF01550000AD8B496
:103BB000AFEF1EF01550010AD8B4B3EF1EF0155048
:103BC000020AD8B4B7EF1EF01550030AD8B4BBEF01
:103BD0001EF01550040AD8B488EF1EF01550000AE4
:103BE000D8B4BCEF1EF01550010AD8B4C0EF1EF0D7
:103BF0001550020AD8B4C4EF1EF01550030AD8B409
:103C0000C8EF1EF01550040AD8B4C9EF1EF01550C5
:103C1000050AD8B4CCEF1EF012009E96C580152A76
:103C20001200E20EC96E152A1200770EC96E152A0F
:103C30001200020EC96E152A12009E96C580152A22
:103C40001200E20EC96E152A1200790EC96E152AED
:103C50001200000EC96E152A12009E96C580152A04
:103C60001200E20EC96E152A12007A0EC96E152ACC
:103C7000120017BC03D0DAC1E8FF04D01750E844A3
:103C8000E8441F09E8CFC9FF152A12009E96C58097
:103C9000152A1200E20EC96E152A120011BA03D0BD
:103CA00011BC01D003D0050E146E3ED00101D667C1
:103CB0005EEF1EF0100EC96E60EF1EF0D6C1C9FF98
:103CC000152A1200D7C1C9FF152A1200D8C1C9FF91
:103CD000152A1200D9C1C9FF152A1200C584152A58
:103CE0001200FF0E156E1A9E12009E96C580152AB0
:103CF0001200E20EC96E152A1200760EC96E152A40
:103D00001200C584152A1200FF0E156E1A9E1200AD
:103D1000C584142A156A12009E96C580152A1200C1
:103D2000E20EC96E152A12007B0EC96E152A12000A
:103D300011AA04D0230EC96E152A12001C0EC96EDA
:103D4000152A12009E96C580152A1200E20EC96E31
:103D5000152A12007C0EC96E152A1200E9D79E960C
:103D6000C580152A1200E20EC96E152A12007D0EBA
:103D7000C96E152A1200DCD79E96C580152A12003E
:103D8000E20EC96E152A12007E0EC96E152A1200A7
:103D9000CFD7C584152A1200FF0E156E1A9E120089
:103DA0001550FF0AD8B48EEF1FF0390EC86E800E82
:103DB000C76E280EC66E000EC56E1450000AD8B429
:103DC000E9EF1EF01450010AD8B4FDEF1EF08EEF9B
:103DD0001FF01550000AD8B43BEF1FF01550010A30
:103DE000D8B43FEF1FF01550020AD8B449EF1FF0C6
:103DF0001550030AD8B44CEF1FF01550000AD8B480
:103E000052EF1FF01550010AD8B456EF1FF01550AD
:103E1000020AD8B460EF1FF01550030AD8B463EF5C
:103E20001FF01550040AD8B469EF1FF01550050AA9
:103E3000D8B46CEF1FF01550060AD8B472EF1FF01B
:103E40001550070AD8B475EF1FF01550080AD8B4FA
:103E50007BEF1FF01550090AD8B47EEF1FF0155004
:103E60000A0AD8B484EF1FF015500B0AD8B487EFB4
:103E70001FF08EEF1FF09E96C5808DEF1FF016B0DD
:103E800004D04E0EC96E8DEF1FF0500EC96E8DEF2F
:103E90001FF0C5848DEF1FF0142AFF0E156E1280DF
:103EA0008EEF1FF09E96C5808DEF1FF016B004D0E8
:103EB0004F0EC96E8DEF1FF0510EC96E8DEF1FF0C2
:103EC000C5868DEF1FF0C9CF21F0C59AC5888DEF4B
:103ED0001FF0C5868DEF1FF0C9CF22F0C59AC588A7
:103EE0008DEF1FF0C5868DEF1FF0C9CF23F0C59A67
:103EF000C5888DEF1FF0C5868DEF1FF0C9CF24F068
:103F0000C58AC5888DEF1FF0C5848DEF1FF0FF0EA9
:103F1000156E12861A9C8EEF1FF0152A120012B031
:103F200012D012B213D012B414D012A6120007B0DD
:103F30001200129621C025F022C026F023C027F0DF
:103F400024C028F0120012901282120012921284E1
:103F5000120000011550FF0A04E11294156AD0EC1A
:043F60001EF012003D
:10BF0000E844F926000C160C2B0C3F0C520C640C68
:10BF1000760C860C960CA50CB30CC10CCF0CDC0C6B
:06BF2000E80CF40C000C1B
:00000001FF
